:100000009DC1B7C1B6C1B5C1B4C194C4B2C1B1C17B
:10001000B0C1AFC1BDC4ADC1ACC1ABC1B8C4B7C440
:10002000B5C4A7C1A6C1A5C1A4C1D3C5A2C1A1C160
:10003000A0C19FC1456E64652064657220466168F9
:100040006E656E7374616E676500312E31202863B2
:1000500029323030392D32303137206D61747A6574
:1000600074726F6E69637300000000000000000688
:100070000004080D8011EE840FEC880DEA8C0BE76C
:10008000900AE59408E29807DF9C05DDA004DAA554
:1000900003D7A802D4AC02D0B001CDB401CAB800D5
:1000A000C6BC00C3BF00BFC300BCC600B8CA01B411
:1000B000CD01B0D002ACD402A8D703A5DA04A0DDEC
:1000C000059CDF0798E20894E50A90E70B8CEA0D9F
:1000D00088EC0F84EE1180F0137BF21577F418731F
:1000E000F51A6FF71D6BF82067FA2263FB255FFC9A
:1000F000285AFD2B57FD2F53FE324FFE354BFF394B
:1001000047FF3C43FF4040FF433CFF4739FE4B3530
:10011000FE4F32FD532FFD572BFC5A28FB5F25FA6B
:100120006322F86720F76B1DF56F1AF47318F277E6
:1001300015F07B13EE8011EC840FEA880DE78C0B31
:10014000E5900AE29408DF9807DD9C05DAA004D761
:10015000A503D4A802D0AC02CDB001CAB401C6B880
:1001600000C3BC00BFBF00BCC300B8C600B4CA0116
:10017000B0CD01ACD002A8D402A5D703A0DA049C6C
:10018000DD0598DF0794E20890E50A8CE70B88EA22
:100190000D84EC0F80EE117BF01377F21573F418D9
:1001A0006FF51A6BF71D67F82063FA225FFB255A7B
:1001B000FC2857FD2B53FD2F4FFE324BFE3547FFDA
:1001C0003943FF3C40FF403CFF4339FF4735FE4B7E
:1001D00032FE4F2FFD532BFD5728FC5A25FB5F2283
:1001E000FA6320F8671DF76B1AF56F18F47315F2B0
:1001F0007713F07B11EE800FEC840DEA880BE78C0F
:100200000AE59008E29407DF9805DD9C04DAA00374
:10021000D7A502D4A802D0AC01CDB001CAB400C6A3
:10022000B800C3BC00BFBF00BCC300B8C601B4CA9D
:1002300001B0CD02ACD002A8D403A5D704A0DA0542
:100240009CDD0798DF0894E20A90E50B8CE70D88A7
:10025000EA0F84EC1180EE137BF01577F21873F43B
:100260001A6FF51D6BF72067F82263FA255FFB28EC
:100270005AFC2B57FD2F53FD324FFE354BFE3947AD
:10028000FF3C43FF4040FF433CFF4739FF4B35FEF7
:100290004F32FE532FFD572BFD5A28FC5F25FB6381
:1002A00022FA6720F86B1DF76F1AF57318F47715AB
:1002B000F27B13F053746F72696E6720454550529C
:1002C0004F4D20200053746F726564202020202041
:1002D00020202020200056462053696E757320444C
:1002E000726976650A00467265712020562F487A39
:1002F0002020416D70200052656164696E67204561
:100300004550524F4D2020005265616420446F6E6D
:10031000652020202020202000502020204920205F
:100320002044202020204454200046726571202063
:10033000562F487A2020416D7020000011241FBEE6
:10034000CFEFD4E0DEBFCDBF11E0A0E0B1E0E0E947
:10035000F2E102C005900D92A032B107D9F721E079
:10036000A0E2B1E001C01D92AC33B207E1F71CD5A9
:100370008DC746CECF93DF93DC01FB01E9011A82E2
:100380001B821C821D82198218829F838E8379872B
:1003900068875B874A878FEF9FE7BD01AED67D8771
:1003A0006C879F01442737FD4095542F61E070E032
:1003B0008FEF9FE7D7D62E873F87488B598BDF91EA
:1003C000CF910895CF92DF92EF92FF920F931F93F8
:1003D000CF93DF938B01FA019C01261B370B848599
:1003E00095858217930784F0919581959109281737
:1003F00039076CF086819781289FE001299FD00DF5
:10040000389FD00D112405C0CFEFDFE702C0C1E057
:10041000D0E8442737FD4095542F82819381A481F1
:10042000B581280F391F4A1F5B1F86859785A089D4
:10043000B18982179307A407B50764F48283938375
:10044000A483B583CC24C394D12CEE24EA949FE7F3
:10045000F92E20C0B095A095909581959F4FAF4FF4
:10046000BF4F281739074A075B075CF482839383E1
:10047000A483B583CC24CA94DC2CE12C80E8F82E2C
:1004800009C02283338344835583A085B18591D6E7
:100490006B017C0180819181801B910BA285B385CA
:1004A0008A9F90018B9F300D9A9F300D11241183EC
:1004B0000083BE01882777FD8095982F6C0D7D1DE8
:1004C0008E1D9F1D8901222717FD2095322F600F59
:1004D000711F821F931F20E031E040E050E042D6C0
:1004E000C901DA01813020E892072FEFA207B20795
:1004F00024F481E090E8AFEFBFEFAC01BD014115FE
:1005000080E858076105710524F04FEF5FE760E070
:1005100070E0CA01DF91CF911F910F91FF90EF9092
:10052000DF90CF900895FC0112821382148215820D
:10053000089584B1817F84B98AB187798AB9089591
:10054000CF93C82FA82FA295AF70B0E0A45FBE4F85
:100550008C91D2D3CF70EC2FF0E0E45FFE4F80811E
:10056000CF91CAC3CF93C82F892FEADF8C2FCF91A9
:10057000E7CF80E2C1C3DF92EF92FF920F931F9308
:10058000CF93DF934AE050E060E071E022D68093A1
:100590003B01E0E0F1E001900020E9F73197E05005
:1005A000F140DE2E80E0E82E81E0F82EC0E0D0E0C1
:1005B0008F011127015011090AC0C017D10711F48A
:1005C0008EE29AD3F70181917F0196D32196CD15C2
:1005D000A0F3DF91CF911F910F91FF90EF90DF90EB
:1005E0000895FB01DA0190911E01981710F0108216
:1005F00011C090911E01482F50E02FEF30E0291BD1
:1006000031094217530744F080911E01880F8095ED
:1006100080838FEF8C93089590911E01282F291BC2
:10062000208390911E01980F9C93089589B1809525
:100630008770089561E080E052D384EB92E078D334
:10064000F89477DFF999FECF60911E0188E090E081
:10065000ECD5F999FECF682D87E090E0E6D5F999C1
:10066000FECF672D86E090E0E0D5F999FECF60914E
:100670002C0170912D0184E090E0E5D5F999FECF31
:1006800060912E0170912F0182E090E0DCD5F99904
:10069000FECF609130017091310180E090E0D3D5C0
:1006A000F999FECF2CE0922A78948FEF99E628E111
:1006B000815090402040E1F700C0000061E080E000
:1006C0000ED385EC92E034D38FEF99E628E1815088
:1006D00090402040E1F700C00000A8CFEF92FF92C9
:1006E0000F931F93CF93DF9305D389E193E020D33A
:1006F000109221019BDF8111FDCF00E098ECF92ED3
:10070000C1E0D0E028E0E22E91DF182F833009F419
:10071000B0C030F4813059F0823009F0ACC014C060
:10072000843009F464C0853009F0A5C0A5C080916B
:1007300021018F5F8093210180912101843008F491
:100740009BC01092210198C0809121018130C1F09D
:1007500030F0823051F1833009F08EC03BC080917F
:100760002C0190912D011816190624F0D0932D011B
:10077000C0932C0180912C0190912D0101974AC0CA
:1007800080912E0190912F011816190624F0D09314
:100790002F01C0932E0180912E0190912F0101977E
:1007A00090932F0180932E0167C08091300190912A
:1007B00031011816190624F0D0933101C09330018D
:1007C0008091300190913101019790933101809394
:1007D000300152C080911E01815080931E01809192
:1007E0001E01883008F048C0E0921E0145C080918B
:1007F00021018130A1F028F0823001F18330E1F550
:100800002CC080912C0190912D0180912C01909110
:100810002D01019690932D0180932C012DC0809184
:100820002E0190912F0120912E0130912F012F5FE9
:100830003F4F30932F0120932E011EC08091300135
:100840009091310120913001309131012F5F3F4F64
:1008500030933101209330010FC080911E018F5FD2
:1008600080931E0180911E01893C30F0F0921E01A0
:1008700003C0E0DE01C000E0409130015091310141
:1008800060912E0170912F0180912C0190912D018A
:1008900026E231E06FDDCADE8823A1F00F5F0A3067
:1008A00050F42FEF8DEE92E0215080409040E1F720
:1008B00000C0000007C08FE39CE90197F1F700C07A
:1008C00000000BE061E080E00AD280912C01909161
:1008D0002D0148DE80912E0190912F0143DE809101
:1008E0003001909131013EDE44DE80911E0128DE10
:1008F00040DEE0912101F0E0E059FF4F849161E09A
:10090000EED18FE19EE40197F1F700C000001530B1
:1009100009F0FACE10922101EBD18AE293E008D2DD
:1009200085DE8111FDCFDF91CF911F910F91FF9057
:10093000EF9008951F920F920FB60F9211242F93EC
:100940003F934F935F936F937F938F939F93AF9357
:10095000BF93EF93FF9389B18095881F8827881FE5
:1009600080FB91F8E6DD8CE0982AFF91EF91BF9132
:10097000AF919F918F917F916F915F914F913F9137
:100980002F910F900FBE0F901F90189518951895E6
:100990001F920F920FB60F921124CF92DF92EF9217
:1009A000FF921F932F933F934F935F936F937F9388
:1009B0008F939F93AF93BF93EF93FF93CF93DF9367
:1009C00000D0CDB7DEB7892D8C70843011F1B1DD48
:1009D00081EB84BD92EB909380008093B0001092E5
:1009E000B3001092880017BC8FEF8093B4008093FF
:1009F0008A0088BD80E286BBB59BFECF892D837FB0
:100A000014E0912E982A84B18E6084B98AB18866E8
:100A10008AB9282C312C8091380190913901820DAE
:100A2000931D909339018093380180913801909102
:100A300039018115904C48F080913801909139012D
:100A4000905C909339018093380120913801309166
:100A50003901232F3327F901EE0FFF1FE20FF31F98
:100A6000EC58FF4F9F012F5F3F4F6491CF010296DB
:100A7000F90191FC04C03491FC01449103C04491FC
:100A8000FC013491649EA0011124E52EE694639E3E
:100A900090011124F32EF694669EC0011124892F33
:100AA000869510E8AE014F5F5F4FBE016E5F7F4FCE
:100AB000F12FF81B8F2F95DD8A8187BD898188BD35
:100AC000AE014F5F5F4FBE016E5F7F4F812F8E196A
:100AD00088DD8A8180938800898180938A00AE01B5
:100AE0004F5F5F4FBE016E5F7F4F812F8F1979DDA2
:100AF0008A818093B30089818093B400809123011F
:100B00008F5F80932301883C08F449C090FE13C096
:100B100020913A01C0903A0130E0AFEFB0E03DD310
:100B2000BB27A92F982F872F46E251E0682D70E050
:100B300049DC882E8C0C682D80E09BE470E0C9D2E3
:100B40009B0140E050E066ED7CED81E090E0E8D272
:100B50003093250120932401C9016AE070E0B9D2E5
:100B6000CB01789EB001799E700D112480E090E059
:100B7000611571058105910551F0663F29E0720705
:100B80008105910524F066EF79E080E090E02AE0AD
:100B900030E040E050E0E6D2622E109223010F9048
:100BA0000F90DF91CF91FF91EF91BF91AF919F9106
:100BB0008F917F916F915F914F913F912F911F91F5
:100BC000FF90EF90DF90CF900F900FBE0F901F908F
:100BD000189578941F920F920FB60F9211242F93AD
:100BE0008F939F9390FE22C080917C00843619F0F1
:100BF0008536B1F40DC020913A018091790090E0E2
:100C0000820F911D9595879580933A0185E609C0DD
:100C10008091790090E0870D911D95958795782EAC
:100C200084E680937C008EED80937A009F918F9173
:100C30002F910F900FBE0F901F901895289A00C00B
:100C4000289808951F93CF93DF931F92CDB7DEB7F7
:100C5000662311F02C9A01C02C982D9897B19F60B3
:100C600097B918B1107F982F92959F70912B98B9D2
:100C70008983E4DF89818F70812B88B9DFDF1F6072
:100C800018B90F90DF91CF911F9108952C982D9A4C
:100C900087B1807F87B9289A00C086B1289800C0A4
:100CA000289A00C096B128989F708295807F892BE2
:100CB0000895ECDF87FDFDCF88E090E00197F1F724
:100CC000E5CFCF93C82FF5DF60E08C2FCF91BACF5F
:100CD000CF93C82FEEDF61E08C2FCF91B3CF61119E
:100CE00002C0805801C08054ECCFE3DF90E008954B
:100CF00081E0E7CF82E0E5CFCF93C82FDADFCA30BB
:100D000041F4803410F480E401C080E08058CF9139
:100D1000D8CF61E08C2FCF9195CFCF93DF93EC01AB
:100D200001C0EADF89918111FCCFDF91CF91089555
:100D3000CF93DF93EC0101C0DFDFFE0121968491A8
:100D40008111FACFDF91CF9108951F93CF93DF9355
:100D5000182F97B19F6097B9249A259A209AE0E0BE
:100D6000FAEF3197F1F7419A409A68DFE0E0FEE44C
:100D70003197F1F763DFC0E0D1E0FE013197F1F781
:100D80005DDFFE013197F1F7409858DF2197F1F7C9
:100D900088E297DF88E095DFABDF86E092DF812F86
:100DA000DF91CF911F918DCFF894612C10923A0171
:100DB00088248394109221018FE087B985B1817FC7
:100DC00085B98BB187798BB98AB1887F8AB98BB1A4
:100DD00087698BB98CE0B9DF8DDF86ED92E0A8DF03
:100DE00080E38ADF21E024BD82E0809380002093AD
:100DF000B0008FEF90E0909387008093860016BC40
:100E000083E090E0909385008093840085E0809358
:100E1000B20025BD81E1809381002093B10081E380
:100E20006BDF80E880936D0084E08093680082E34C
:100E300063DF86E980937A0080E380937E0084E616
:100E400080937C0010927B0086EC80937A0071DBAB
:100E50002FEF83EC99E0215080409040E1F700C0F3
:100E600000008EED80937A0083E346DF26E231E0D6
:100E700040E150E068E070E080E690E07BDA84E3F7
:100E80003BDFE89490F8E89491F82CE0922A85E30F
:100E900033DF89B18095881F8827881F80FB91F8F0
:100EA0004C9903C0689490F802C0E89490F887E2E7
:100EB00086BB80E280936F0086E31EDF8FEF99E6AA
:100EC00028E1815090402040E1F700C0000061E03F
:100ED00080E005DF87EF92E02BDF88E090E098D19B
:100EE00080931E0180911E01883018F488E0809361
:100EF0001E0187E090E08CD1882E86E090E088D1BA
:100F0000782E84E090E08CD190932D0180932C0179
:100F100082E090E085D190932F0180932E0180E0B4
:100F200090E07ED190933101809330018FEF99E66C
:100F300028E1815090402040E1F700C0000061E0CE
:100F400080E0CDDE88E093E0F3DE8FEF99E628E1E4
:100F5000815090402040E1F700C0000067DB87E34C
:100F6000CBDEC6DE8EE0ADDE86EE92E0E1DE78948A
:100F70006BE0D62E0FEF10E059DB90FC3FC08230C3
:100F8000A9F018F48130F1F505C08330C9F184303F
:100F9000C9F51FC0809121018F5F8093210180914D
:100FA0002101823088F1109221012EC0809121010F
:100FB000882319F0813041F506C0811002C08824D1
:100FC00083948A9421C0711002C0772473947A9418
:100FD0001BC080912101882319F08130A9F407C03A
:100FE0008FEF881202C05EEF852E83940DC09FEFB5
:100FF000791202C04EEF742E739406C0833011F440
:101000006DDB02C01092220111DB8823C9F08091B0
:1010100022018F5F809322018A3050F42FEF8DEEF2
:1010200092E0215080409040E1F700C0000008C0ED
:101030008FE39CE90197F1F700C00000D0922201F4
:1010400061E080E04CDE809124019091250193DAEB
:1010500090DA61E086E043DE872D90E08CDA89DA71
:1010600088DA61E08CE03BDE24E6629EC001112458
:10107000B8012FD0CB014AE050E060E071E0A9D088
:1010800080933B01E0E0F1E001900020E9F7319727
:10109000E050F140CE2E30E0E32E31E0F32EE701B8
:1010A00002C0899129DE8C2F8E198C15D0F385E230
:1010B00023DE5FDAE0912101F0E0E259FF4F8491F5
:1010C00061E00DDE8FE19EE40197F1F700C00000C2
:1010D00053CFAA1BBB1B51E107C0AA1FBB1FA617FA
:1010E000B70710F0A61BB70B881F991F5A95A9F7D1
:1010F00080959095BC01CD01089597FB072E16F4BD
:10110000009406D077FD08D0E4DF07FC05D03EF45C
:10111000909581959F4F0895709561957F4F0895A3
:10112000A1E21A2EAA1BBB1BFD010DC0AA1FBB1FEB
:10113000EE1FFF1FA217B307E407F50720F0A21B5D
:10114000B30BE40BF50B661F771F881F991F1A94CA
:1011500069F760957095809590959B01AC01BD01F4
:10116000CF010895052E97FB16F4009406D057FD85
:101170000CD0D6DF07FC09D07EF490958095709551
:1011800061957F4F8F4F9F4F0895509540953095B3
:1011900021953F4F4F4F5F4F0895A29FB001B39FDE
:1011A000C001A39F01D0B29F700D811D1124911D1C
:1011B0000895B7FF04C003D0821B930B0895EDDFA1
:1011C000A59F900DB49F900DA49F800D911D11249B
:1011D0000895FB019F01E8944230BCF04532ACF425
:1011E0004A3029F497FB1EF4909581959F4F642F08
:1011F00077276FDF805D8A330CF0895D8193CB01A7
:101200000097A9F716F45DE251931082C9011EC040
:10121000F999FECF92BD81BDF89A992780B50895BE
:10122000A8E1B0E042E050E023C0262FF999FECFBC
:101230001FBA92BD81BD20BD0FB6F894FA9AF99AF3
:101240000FBE01960895F1DF272FF0CFDC01FC01DE
:10125000672F71917723E1F7329704C07C916D93EA
:1012600070836291AE17BF07C8F30895DC01CB010C
:10127000FC01F999FECF06C0F2BDE1BDF89A3196A6
:1012800000B40D9241505040B8F70895F894FFCF44
:101290003030303030303030303030303031323348
:1012A000343536373839414243444546000014004E
:00000001FF
